:0400000002002432A4
:01000B0032C2
:0100130032BA
:03001B000200954B
:100023003279207A60E4F709DAFC758910D28ED22E
:10003300AFD2AB75810875300712006020E00F3036
:10004300E1F71530E530B402F075301480EB05327A
:10005300753300E532640770E0F53280DCE420B4E8
:100063000C12008030B4FD120080D2E02230B501C2
:100073002212008030B5FD120080D2E1227F70E4AD
:100083001470FDDFFB227F00DFFE227E0A1180DE7B
:10009300FC22C0E0C0D0E8C0E0E5316005153102C4
:1000A30001DA853031E532B40012E533780020E01F
:1000B3000278FF889088A088800201D8B4011AE5ED
:1000C30033785579AA7A5520E00678AA79557AAA21
:1000D300889089A08A800201D8B40227E533B4034B
:1000E300047400F53378FF79FF7AFFB400027800D7
:1000F300B401027900B402027A00889089A08A8050
:100103000201D8B40330E533B418047400F533782E
:10011300FE79FF7AFFFBEB600CE8D333F8E933F9A0
:10012300EA13FADBF4889089A08A80E5310303544B
:100133003FF5310201D8B40431E533B41804740037
:10014300F53378FF79FF7AFEFBEB600CEAD333FAE1
:10015300E913F9E813F8DBF4889089A08A80E53184
:10016300030303541FF5310201D8B40532E533B458
:1001730008047400F53378FE79FE7A7FFBEB600E9A
:10018300E8D333F8E9D333F9EAD313FADBF28890EF
:1001930089A08A80E5310303543FF5310201D8B4C5
:1001A3000633E533B408047400F533787F797F7A36
:1001B300FEFBEB600EEAD333FAE9D313F9E8D3136A
:1001C300F8DBF2889089A08A80E531030303541F8A
:1001D300F5310201D80533C28FD0E0F8D0D0D0E09A
:0101E30032E9
:00000001FF
